:0200000480007A
:100000006F00C004732F2034930F8000630AFF0336
:10001000930F90006306FF03930FB0006302FF038A
:10002000170F0080130F0FFE63040F0067000F000F
:10003000732F203463540F006F004000136E9E53E3
:10004000171F00002320CFFD6FF09FFF732540F1A5
:100050006310050073251030635805000F00F00F82
:10006000130E100073000000130E00009702000032
:10007000938282F973905230735020307350303035
:1000800073504030970200809382C2F7638C020065
:10009000739052109302B01A739022307323203061
:1000A000E39E62F873500030970200009382420191
:1000B00073901234732540F173002030B70001FFB4
:1000C000938000F093E1F0F0930EF0F0130E200017
:1000D0006394D11DB710F00F938000FF93E1000FE0
:1000E000B71EF00F938E0EFF130E30006396D11BD8
:1000F000B700FF009380F00F93E1F070B70EFF00A0
:10010000938EFE7F130E40006398D119B7F00FF065
:100110009380F00093E1000FB7FE0FF0938EFE0F77
:10012000130E5000639AD117B70001FF938000F0BF
:1001300093E0000FB70E01FF938E0EFF130E6000C9
:10014000639CD01513020000B710F00F938000FFDE
:1001500093E1000F138301001302120093022000A9
:10016000E31452FEB71EF00F938E0EFF130E7000B5
:100170006314D31313020000B700FF009380F00F45
:1001800093E1F070130000001383010013021200CA
:1001900093022000E31252FEB70EFF00938EFE7F03
:1001A000130E8000631AD30F13020000B7F00FF094
:1001B0009380F00093E1000F130000001300000093
:1001C000138301001302120093022000E31052FE79
:1001D000B7FE0FF0938EFE0F130E9000631ED30B2D
:1001E00013020000B710F00F938000FF93E1000F9F
:1001F0001302120093022000E31652FEB71EF00F06
:10020000938E0EFF130EA0006398D1091302000015
:10021000B700FF009380F00F1300000093E1F0F0AF
:100220001302120093022000E31452FE930EF0FF1B
:10023000130EB0006392D10713020000B7F00FF065
:100240009380F000130000001300000093E1000F02
:100250001302120093022000E31252FEB7FE0FF0C9
:10026000938EFE0F130EC0006398D1039360000FAE
:10027000930E000F130ED0006390D003B700FF0061
:100280009380F00F13E0F070930E0000130EE00067
:100290006314D001631CC0010F00F00F63000E0057
:1002A000131E1E00136E1E00730000000F00F00FDF
:1002B000130E100073000000731000C00000000057
:0402C000000000003A
:1010000000000000000000000000000000000000E0
:1010100000000000000000000000000000000000D0
:1010200000000000000000000000000000000000C0
:1010300000000000000000000000000000000000B0
:081040000000000000000000A8
:040000058000200057
:00000001FF
